:020000040800F2
:1000000040180020C9000008C90F00085507000863
:1000100000000000000000000000000000000000E0
:10002000000000000000000000000000FF100008B9
:1000300000000000000000004D130008B11300088C
:10004000DB00000800000000DB000008DB00000807
:10005000DB000008DB000008DB000008DB00000814
:1000600000000000DB000008D9030008F5040008C8
:10007000DB000008DB000008DB00000800000000D7
:10008000DB0000081116000800000000DB0000087B
:10009000DB000008E1150008DB000008DB000008B9
:1000A000DB000008F7100008DB00000875180008E6
:1000B000351900080348854600F0B8F800480047A5
:1000C00019200008401800200448804704480047D1
:1000D000FEE7FEE7FEE7FEE7FEE7FEE76D15000838
:1000E000B500000830B50B4601460020202201244F
:1000F00009E00D46D5409D4205D31D469540491B5C
:100100002546954040191546521E002DF1DC30BDA4
:1001100070B500242546002801DA01244042002958
:1001200001DA01254942FFF7DDFFAC4200D0404231
:10013000002C00D0494270BDF8B5002425460029A6
:1001400004DA0E46012400214042B141002B04DABA
:100150001E46002352420125B34100F036F88C467A
:1001600017461E46AC4203D0002540428D41AC46A6
:10017000002C02D0002657429E4161463A46334643
:1001800001B0F0BD10B5202A04DB0846203AD0406B
:10019000002110BD0B46D340D0402024A21A91402C
:1001A0000843194610BDD2B201E00270401C491E3E
:1001B000FBD270470022F6E710B513460A46044604
:1001C0001946FFF7F0FF204610BDF0B51FB40646F4
:1001D000002082B005464024019100901BE0019967
:1001E00022460F463046FFF7CDFF049A059B801A42
:1001F000994110D310461946224600F029F8361AC4
:100200008F410197224601200021009F00F020F835
:1002100038184D4100902046641E0028DFDC019B09
:1002200000982946324607B0F0BD0000064C012573
:10023000064E05E0E36807CC2B430C3C984710348E
:10024000B442F7D3FFF73AFF681D0008881D000885
:1002500010B5202A04DB0146203A9140002010BD51
:10026000914020239C1A0346E3401943904010BD5F
:1002700070B5002100BF4848806804221040800803
:1002800000287DD100BF444B1B6C9BB21946434BE9
:1002900018680122C307DB0F002B0ED0404B1984D6
:1002A000404A1B8C404CA34203DA01233F4C23609D
:1002B0005CE000233D4C236058E03A4B0340394C4E
:1002C000A34206D13A4B1B885B18394C2380394A2C
:1002D0004CE0384B0340374CA34225D1344B5B886C
:1002E0005B18334C6380344B1B685B1C324C2360BF
:1002F00023461B68082B15DB2D4C2388DC17640F65
:10030000E418E410264D2035EC80294C6388DC1776
:10031000640FE418E4102C810023254C23806380B3
:10032000254C2360254A21E0244B0340234CA34263
:1003300004D11B4B20335981214A17E0214B034044
:10034000204CA34204D1164B203399811E4A0DE064
:100350001E4B03401D4CA34208D1114B2033D981C1
:100360001B4B5C8B0E4B20331C82012200BF5303BE
:100370005B0B094CA36200BF00BF23469B6800E0F3
:1003800008E0144C23401B1D034CA36000BF034B2B
:100390001A6000BF002070BD00240140180000203A
:1003A0000C0500208000001CDC05000094000020EB
:1003B0006C01002000010020140000200002002435
:1003C000000001C000000140000002C4000002441F
:1003D000A0F7FF1FE8FFFF7F70B54248C06A401CCE
:1003E0004049C86200BF40480068202108404009D9
:1003F000002866D03B4800683A49096B40183949E3
:1004000008600846016B443000F0A4F800BF2020CB
:100410003549486000BF33484430817A8907C90FA5
:10042000002945D100F0CCF804462F4802214A1E8D
:100430002E4B9A5C825853085B004A1E2B4DAA5CD7
:10044000835000BF024602232649443108268E5FAE
:100450000D68A81900BF591E244D695C8918C86031
:1004600000BF1046022122464B1EEB5C1B185B6846
:100470001B0C1B0413434D1E1C4E755D2D186B6029
:1004800000BF00BF4A1E33469A5C825801231A43BC
:100490004B1E3546EB5CC25000BF1248046300BFE0
:1004A00013488068802108431149886000BF08E034
:1004B00000200C4908630846007B02218843094953
:1004C000087300BF08480068012149020840400A3B
:1004D000002805D000BF08460349486000BF00BFA0
:1004E00070BD00008C01002000000240CE1C0008FE
:1004F000003801401548C06A401C1449C86200BF5A
:1005000013480068012149030840400B00280DD022
:1005100000BF08460E49486000BF00200B49086331
:100520000846007B022188430849087300BF084839
:100530000068012149040840400C002805D000BF94
:1005400008460349486000BF00BF7047DC01002037
:100550000000024010B502460B46002B01D11846A0
:1005600010BD0820105EC1180420105E884202DC15
:100570000420105E091A907A40084000907208B278
:1005800010810620105E884207D10020D0801081A3
:10059000907A0224A043801C90721846E0E708B5C8
:1005A00000210AE00022009203E000BF009A521CE2
:1005B0000092009A182AF8DB491C8142F2DB08BD40
:1005C00070B504460825655F0626A65FB54201DAC8
:1005D000701B70BDB54203DD0420205E401BF8E7B0
:1005E00000BFA07AC007C00F002803D00420205EFF
:1005F000401BEEE7204600F003F9002801D0002060
:10060000E7E70020E5E70000084B1968084B9A6906
:10061000064B1B68994203D0044B1968044B9A6936
:10062000044B53431B14C81A7047000030000020CD
:1006300000E000E05505000002480068401C014948
:1006400008607047E800002010B5064800681021D7
:10065000084304490860002000F006F800F018F88C
:10066000002010BD0020024070B5044600F04AF89A
:1006700006467D21C900FFF735FD054600F04AF822
:1006800000222146501E00F033F8002070BD00000B
:1006900008B500BF154880690121084313498861E6
:1006A00008468069C007C00F009000BF00BF00BFB0
:1006B0000846C069090408430C49C8610846C06976
:1006C00009040840009000BF00BF00221146501FDF
:1006D00000F00EF800221146901E00F009F80022EA
:1006E0001146501E00F004F808BD00000010024042
:1006F00070B504460D4616462946204600F066FCB5
:1007000070BD00000148006870470000E400002050
:100710007047000070B504462546681E09498842A6
:1007200001D901200CE0681E074948610321081F18
:1007300000F04CFC0020044988610720086100207B
:1007400070BD0000FFFFFF0000E000E010B5FFF704
:10075000DFFF10BD00BFFEE7F8B504460E461746A2
:100760001D46502200212046FFF71DFD002E05D01A
:100770003A4631462046383001F06FF9002D05D059
:10078000294620464430069A01F067F90020F8BD5A
:1007900070B5044621461248FFF7BAFC11490860BB
:1007A000FFF7B0FF05460E49FFF79CFC0E490860B5
:1007B00021460E480068FFF795FC0D4908600B487C
:1007C000002302680B480F21FFF7B6FC0A49088096
:1007D00004480068643009490860002070BD0000CA
:1007E00040420F002800002020000020E4000020EC
:1007F000240000200000404234000020300000208F
:100800000146887A8007C00F7047000010B5044683
:100810000249002000F004F8002010BD5400002020
:1008200030B50246054B186A8300044C2434E1506D
:10083000024B1B6A5B1C243C236230BDAC060020CB
:1008400008B5054949690143034A5161114649699F
:100850000140009100BF08BD0010024008B50549E5
:1008600089690143034A91611146896901400091F8
:1008700000BF08BD00100240F0B502460B4600263E
:10088000002162E00124B44018682040014600299C
:100890005AD0586814680D464D436F00ED19AC43AB
:1008A0000D464D4345432C43146000BF5868012852
:1008B00002D0586802280DD1986894680D464D43BF
:1008C0006F00ED19AC430D464D4345432C439460F6
:1008D00000BF00BF1869D4680D464D436F00ED1985
:1008E000AC430D464D4345432C43D46000BF58688C
:1008F000022829D1FF2911D85869146A0D464D43A1
:100900004D434D432F017D1BAC430D464D434D439D
:100910004D4345432C43146200BF15E05F69080A4C
:1009200040430C0A60430C0A60430401241A506AD5
:10093000A0430C0A64430D0A6C430D0A6C437C43CC
:100940002043506200BF00BF761C1868F0400028AA
:1009500098D15868012802D05868022809D1DC686B
:10096000186855688543074667433D43556000BF97
:1009700000BF0120F0BD024610690840884201D145
:10098000012070470020FCE701460869704781623A
:10099000704781617047000070B504467D25ED0009
:1009A00029462046FFF79EFB401E0449486100206F
:1009B00088610520086100BF70BD000000E000E014
:1009C00001468868C007C00F012250405040704760
:1009D0000146C868C0B2704701490860704700000E
:1009E000E400002010B5034600220C7B224610468E
:1009F00003242402A0438C682043024610460124AD
:100A0000A402A0434C682043024610460124E4029D
:100A1000A0430C6820430246104601242403A0434F
:100A2000CC8920430246104601246403A0430C698C
:100A30002043024610460124A403A0434C692043EE
:100A4000024610460124E403A0434C6920430246B9
:100A50005A64012010BD026A0A4302627047416C69
:100A60000122D203914341647047816880229143FF
:100A70008160704701688022114301607047416CBA
:100A80000122D203114341647047016801221143DE
:100A90000160704710B50246002313682148824266
:100AA00002D02148824205D118467024A0434C68E8
:100AB000204303461B4882420ED01B4882420BD083
:100AC0001A48824208D01A48824205D01948824208
:100AD00002D01948824206D1184603242402A043BA
:100AE000CC682043034613608868D06200BF088842
:100AF000906200BF0B48824208D00D48824205D068
:100B00000C48824202D00C48824203D1087C106318
:100B100000BF00BF00BF506901242043506100BFE7
:100B2000012010BD002C01400004004000200040C6
:100B3000004001400044014000480140014608696E
:100B4000C007C00F012250405040704770B50246A8
:100B5000012901D1002418E0042901D1012414E065
:100B6000102901D1022410E0402901D103240CE016
:100B7000FF240134A14201D1042406E00124A4028F
:100B8000A14201D1052400E006242346064CE55C81
:100B9000144618342819054DEE5C0425B540046848
:100BA000AC43046070BD0000451D00084C1D0008EA
:100BB00070B50246012901D1002418E0042901D1B1
:100BC000012414E0102901D1022410E0402901D1B0
:100BD00003240CE0FF240134A14201D1042406E0E7
:100BE0000124A402A14201D1052400E006242346E9
:100BF000064CE55C144618342819054DEE5C0825B2
:100C0000B54004682C43046070BD0000451D000819
:100C10004C1D0008F8B506460C4615460027012C69
:100C20000AD0102C0ED0E01FF938002810D00F2168
:100C30000902401A18D111E02946304600F002FAA4
:100C4000074612E02946304600F06AFA07460CE0F3
:100C50002946304600F0CAFA074606E029463046E3
:100C600000F026FB074600E000BF00BF3846F8BD95
:100C7000416370478163704781637047C162704709
:100C80008268024B1A400A4382607047F8BFFFFF38
:100C9000426870239A430A43426070470146C8691C
:100CA00010221040000970470146C8690822104010
:100CB000C00870470146C8692022104040097047AB
:100CC0000146C86940221040800970470146086803
:100CD000102210400009704700B599B0142114A8E3
:100CE000FFF768FA20210CA8FFF764FA182106A87C
:100CF000FFF760FA18216846FFF75CFA012000044C
:100D0000FFF7ACFD002110A80182002015903D489E
:100D100016900020179018A8017014A93A48FFF700
:100D2000B9FE3948FFF7A6FE00213748FFF7A8FFB4
:100D300060200C9000200D900E906B20C0000F9052
:100D400000201090022011900020129013900CAA05
:100D500001212D48FFF75EFF01212B48FFF7F6FE2A
:100D600010212948FFF724FF70200C9000200D90DF
:100D70000E9064200F900CAA10212348FFF74AFF21
:100D800010212148FFF7E2FE50211F48FFF780FFA6
:100D90001D48FFF76AFE0020069007900890142176
:100DA00008A8017100216846C184012040030A900F
:100DB00000200B9006A91448FFF714FE01208004C0
:100DC000FFF73EFD012080030090022001900020EB
:100DD0000290039004900120059069460B48FFF7AC
:100DE0004BFD0120C00300900220019000200290E2
:100DF000039004900320059069460448FFF73CFDEA
:100E000019B000BDB10600000040014000040048D8
:100E100000B599B0142114A8FFF7CCF920210CA833
:100E2000FFF7C8F9182106A8FFF7C4F9182168468A
:100E3000FFF7C0F90120C002FFF710FD002110A844
:100E40000182002015905C4816900020179018A889
:100E5000017014A95948FFF71DFE5848FFF70AFE14
:100E600000215648FFF70CFF01215448FFF7A0FE70
:100E700060200C9000200D900E9051480F900220A1
:100E8000109000201190129013900CAA01214B4851
:100E9000FFF7C0FE01214948FFF758FE0121090371
:100EA0004648FFF785FE60200C90002010900D90C2
:100EB0000E906B20C0000F900CAA012109033F483F
:100EC000FFF7A8FE012109033C48FFF73FFE002081
:100ED0003A498968702291430143384A916000BFC2
:100EE000042011468968C908C9000143916000BF08
:100EF00000BF1046C068402188431146C86000BF4B
:100F000000BF0846C0680121890388431146C860B4
:100F100000BF00211046FFF7BBFE2848FFF7A5FDE4
:100F20000020069007900890502108A80171002128
:100F30006846C184012040030A9000200B9006A956
:100F40001E48FFF74FFD01208004FFF779FC0120C8
:100F50004004FFF775FC012040030090022001903F
:100F600000200290039004900220059069461548E5
:100F7000FFF782FCFF20013000900220019000204A
:100F80000290039004900220059069460920C00653
:100F9000FFF772FC0120C0020090022001900020A7
:100FA0000290039004900220059069460920C00633
:100FB000FFF762FC19B000BDB1060000002C014033
:100FC00059030000000400487047000010B50028D5
:100FD00019DA1A4A03071B0F083B9B089B00D258DB
:100FE0008307DC0EFF23A3409A438B071B0E840765
:100FF000E40EA3401A43114B0407240F083CA40835
:10100000A4001A5118E00E4A03231B02D2188308C9
:101010009B00D2588307DC0EFF23A3409A438B0723
:101020001B0E8407E40EA3401A43054B032424023D
:101030001B198408A4001A5110BD00001CED00E02B
:1010400000E100E070B50246002400230025106A8C
:10105000400840001062136A55689469A408A4000F
:1010600020467026B0430E683043044618460226D8
:10107000B0430E6930430346580840004E68304381
:1010800003461848824208D01748824205D01748C4
:10109000824202D0164882421CD118460826B0432C
:1010A0004E69B6003043034618460426B0438E68A6
:1010B000B600304303462846FF260136B0438E690A
:1010C00030430546284601267602B043CE697600B5
:1010D0003043054655609461C868506300BF136291
:1010E000012070BD002C014000400140004401403F
:1010F00000480140704710B500F03AF910BD704744
:1011000055AA010320000000120101090010000C83
:1011100000100008881D000800900008CCCC55AADB
:10112000F8B504460D460027002600200090206AEE
:10113000102188432062266A60680090A769032115
:101140000902384688430746384607210903884381
:101150002968090208430746304620218843296947
:101160000901084306463046102188436968090191
:10117000084306461948844208D01948844205D0DD
:101180001848844202D0184884421DD1304680213C
:1011900088436969890108430646304640218843EF
:1011A000A9688901084306460121890200988843FD
:1011B000A9698900084300900121C9020098884369
:1011C000E969C9000843009000986060A761204663
:1011D000E968FFF751FD26620120F8BD002C0140AF
:1011E00000400140004401400048014070B5024603
:1011F000002400230025106AFF260136B043106248
:10120000136A5568D469A408A40020467026B04328
:101210000E6830430446184601267602B0430E6934
:101220003602304303461846FF260136B0434E6867
:101230003602304303461A48824208D01948824297
:1012400005D01948824202D0184882421FD1184660
:101250000126F602B0434E69B602304303461846F3
:101260000126B602B0438E68B602304303462846D4
:1012700001263603B0438E693601304305462846C1
:1012800001267603B043CE697601304305465560AA
:10129000D461C868D06300BF1362012070BD000034
:1012A000002C014000400140004401400048014042
:1012B00070B50246002300240025106A012636037B
:1012C000B0431062146A5568D36903263602184683
:1012D000B0430346184607263603B0430E6836026D
:1012E00030430346204601267603B0430E69360399
:1012F00030430446204601263603B0434E68360389
:10130000304304460D48824208D00D48824205D041
:101310000C48824202D00C48824207D1284601265E
:10132000B603B0438E69B601304305465560D361BC
:10133000C868106400BF1462012070BD002C014019
:1013400000400140004401400048014010B5012028
:10135000C0060549486005480068401C034908600C
:10136000FFF7C8FE10BD000000ED00E040000020C7
:1013700010B50548FFF724FB002804D00248FFF70A
:1013800027FB044600BF10BD0030014010B50446E5
:10139000002C05D0012109030448FFF7F8FA04E006
:1013A000012109030148FFF7F4FA10BD00040048C9
:1013B00010B5FFF741F9FFF7C9F910BD10B50120CD
:1013C0005F490968814301435D4A116000BF00BF66
:1013D00010460068C007C00F002803D11E2159A085
:1013E00000F02AFB00BF5D480068012109040843A2
:1013F0005A49086000BF00BF00BF5848006801217B
:1014000049040840400C0028F6D000BF5348406B08
:10141000012108435149486300BF00BF00BF4F4846
:10142000406B0221084040080028F7D010204B49AB
:10143000496BF8229143C2001143484A516300BFEF
:1014400000BF1046406A012108431146486200BFB0
:1014500043480521C90452683D231B049A430304F1
:1014600003400B431A433D4B5A601A46D26A120995
:10147000120103071B0F1A43384BDA6200BF00BF8B
:10148000184600680121090608431946086000BF94
:1014900000BF00BF31480068012149060840400EE6
:1014A0000028F6D000202D494968F02291430143DD
:1014B0002A4A516000BF00BF114649680722120244
:1014C00091430143254A516000BF022011464968FB
:1014D000890889000143516000BF00BF00BF1F4859
:1014E00040680C2108400828F8D11E48FFF754FA3C
:1014F0000420042806D11C490969042211431A4A10
:10150000116105E01849096904229143164A1161E5
:1015100000BF1448FFF760FA00BF1048406B042179
:1015200088430E49486300BF0020096B0022134620
:1015300003229A4091430143084A116300BF10BD42
:10154000002002405372635C4253505F556C7472CA
:1015500061536F6E69632E6300000000001002404B
:1015600001000100006CDC0200E000E019480068A6
:101570000121084317490860084640681649084099
:101580001449486008460068144908401149086039
:10159000084600680121890488430E49086008460E
:1015A00040683F21090488430A4948600846C06AE8
:1015B00000090001C8620846006BFF21143188430E
:1015C000044908630846406B400840004863002017
:1015D00088607047001002400CB8FF08FFFFF6FE5D
:1015E00010B50948FFF7AAFA002806D000BF01206D
:1015F000C0430549086100BF00BF04480079401C92
:10160000C1B20248017110BD004401404C060020E7
:1016100010B50948FFF792FA002806D000BF012054
:10162000C0430549086100BF00BF04488078401CE2
:10163000C1B20248817010BD001000404C0600206D
:1016400070B50121C9030920C006FFF7A0F92021C8
:101650001248FFF79EF900260124002519E0082111
:101660000E48FFF794F90120FEF799FF08210B4877
:10167000FFF78FF90120FEF792FF20210748FFF7BF
:101680007AF9002802D03046204306466006040E50
:101690006D1C082DE3DB304670BD000000040048DF
:1016A00070B505460121C9030920C006FFF771F98D
:1016B00008211148FFF76DF920210F48FFF769F95C
:1016C0000220FEF76CFF0121C9030920C006FFF7C5
:1016D0005EF9422000F012F8002403E0FFF7B0FFAB
:1016E0002855641C042CF9DB0121C9030920C0061C
:1016F000FFF74FF970BD00000004004870B50646C2
:101700000121C9030920C006FFF741F90124002582
:101710001DE008210F48FFF73AF930462040002825
:1017200004D020210B48FFF734F903E020210948B9
:10173000FFF72DF90120FEF732FF08210548FFF7DA
:1017400028F96006040E0120FEF729FF6D1C082D04
:10175000DFDB70BD00040048F8B505460E461746AD
:1017600000F034F8E8B200F00FF8002403E0305D38
:10177000FFF7C4FF641CBC42F9DB0121C903092047
:10178000C006FFF706F9F8BD10B504460121C903EC
:101790000920C006FFF7FDF808210B48FFF7F9F80C
:1017A00020210948FFF7F5F80220FEF7F8FE012195
:1017B000C9030920C006FFF7EAF8C0212143084603
:1017C000FFF79CFF10BD00000004004810B5012188
:1017D000C9030920C006FFF7DCF808210C48FFF711
:1017E000D8F820210A48FFF7D4F80220FEF7D7FEE8
:1017F0000121C9030920C006FFF7C9F84020FFF7FF
:101800007DFF0121C9030920C006FFF7C2F810BD02
:101810000004004810B50121C9030920C006FFF7E4
:10182000B8F808210E48FFF7B4F820210C48FFF75C
:10183000B0F80220FEF7B3FE0121C9030920C0065B
:10184000FFF7A5F88A20FFF759FF0121C9030920F6
:10185000C006FFF79EF820210148FFF79AF810BD57
:10186000000400480120000701494860704700005B
:1018700000ED00E010B52948FFF71CFA002820D041
:101880000121274A1170274A117027494969491CCB
:10189000254A516100BF2149898CC9B208461146C9
:1018A0004968491C51602149214A128888542049BD
:1018B0000988FF2904DA1E490988491C1C4A11803D
:1018C00000BF1648FFF7F0F9002809D000BF082034
:1018D0001249086200BF1448006A401C124908629D
:1018E0000E48FFF7F3F900280BD00C48FFF7D6F9A4
:1018F000002806D000BF10200849086200BF00F091
:101900004FF80648FFF7DCF9002806D000BF40205A
:101910000249086200BF00F057F810BD00380140CE
:10192000BC000020BD0000208C0100201409002014
:10193000AC00002010B51848FFF7BCF91648FFF7B7
:10194000B3F9002809D000BF08201349086200BF7E
:101950001248006A401C114908620F48FFF7B6F9A7
:1019600000280BD00C48FFF799F9002806D000BFDB
:1019700010200949086200BF00F02EF80648FFF762
:101980009FF9002806D000BF40200349086200BF2D
:1019900000F044F810BD000000440040DC010020CD
:1019A00000B50748806A401C0549886205480088E0
:1019B000002803DD01204873FFF754FF00BD00003D
:1019C0008C010020AC0000200248406A401C014904
:1019D000486270478C01002000B50C4805214A1E62
:1019E0000B4B9A5C121852684020801A09490880F3
:1019F0000120094948730846806A401C88620548EE
:101A00000088002801DDFFF72DFF00BD0000024027
:101A1000801A0008AE000020DC01002000B5054857
:101A2000406A401C0349486201208873FFF71AFF8F
:101A300000BD0000DC01002000BFFEE702E008C896
:101A4000121F08C1002AFAD170477047002001E038
:101A500001C1121F002AFBD1704710B5034619605F
:101A600010B298800020D8801881987A40084000F1
:101A70009872987A0224A043801C9872002010BDAE
:101A8000081C304458000000000404040000080052
:101A90000000080000080000000800020406080A10
:101AA0000C0001020304050600C1814001C0804111
:101AB00001C0804100C1814001C0804100C181401E
:101AC00000C1814001C0804101C0804100C181400E
:101AD00000C1814001C0804100C1814001C08041FE
:101AE00001C0804100C1814001C0804100C18140EE
:101AF00000C1814001C0804100C1814001C08041DE
:101B000001C0804100C1814000C1814001C08041CD
:101B100001C0804100C1814001C0804100C18140BD
:101B200000C1814001C0804101C0804100C18140AD
:101B300000C1814001C0804100C1814001C080419D
:101B400001C0804100C1814000C1814001C080418D
:101B500001C0804100C1814001C0804100C181407D
:101B600000C1814001C0804100C1814001C080416D
:101B700001C0804100C1814001C0804100C181405D
:101B800000C1814001C0804101C0804100C181404D
:101B900000C1814001C0804100C1814001C080413D
:101BA00001C0804100C1814000C0C101C30302C225
:101BB000C60607C705C5C404CC0C0DCD0FCFCE0E8D
:101BC0000ACACB0BC90908C8D81819D91BDBDA1AFD
:101BD0001EDEDF1FDD1D1CDC14D4D515D71716D66D
:101BE000D21213D311D1D010F03031F133F3F232DD
:101BF00036F6F737F53534F43CFCFD3DFF3F3EFE4D
:101C0000FA3A3BFB39F9F83828E8E929EB2B2AEABC
:101C1000EE2E2FEF2DEDEC2CE42425E527E7E6262C
:101C200022E2E323E12120E0A06061A163A3A2629C
:101C300066A6A767A56564A46CACAD6DAF6F6EAE0C
:101C4000AA6A6BAB69A9A86878B8B979BB7B7ABA7C
:101C5000BE7E7FBF7DBDBC7CB47475B577B7B676EC
:101C600072B2B373B17170B050909151935352925C
:101C700096565797559594549C5C5D9D5F9F9E5ECC
:101C80005A9A9B5B99595898884849894B8B8A4A3C
:101C90004E8E8F4F8D4D4C8C4484854587474686AC
:101CA0008242438341818040000001CC01D800146E
:101CB00001F0003C002801E401A0006C007801B4B0
:101CC0000050019C01880044060000000400081C2C
:101CD0003044580000000004040400000800000024
:101CE000080000080000000800020406080A0C00B2
:101CF000010203040506081C3044580000000004DB
:101D000004040000080000000800000800000008AB
:101D100000020406080A0C000102030405063F063F
:101D20005B4F666D7D077F6F777C395E7971BF860B
:101D3000DBCFE6EDFD87FFEFF7FCB9DEF9F1004000
:101D4000081C30445800000000040404000008008F
:101D50000000080000080000000800020406080A4D
:101D60000C000102030405060827000800000020FB
:101D7000EC0000003C1A0008F4270008EC000020EA
:101D8000541700004C1A000800000000000000007A
:101D90000000000000000000000000000000000043
:101DA0000000000000000000000000000000000033
:101DB0000000000000000000000000000000000023
:101DC0000000000000000000000000000000000013
:102000000109120102010401040110100000000086
:102010000000000200000600A6B00120FE4908836F
:10202000FF200530FD4B8022FD490090FD48FEF762
:1020300093FB4020FC4B0246FC490090FC48FEF715
:102040008BFBFEF701FB00260020FA49086348637A
:10205000F94888630020C863F848C06A0863F848F4
:1020600000684863F748406A8863F748FEF797FAC4
:10207000FFF7A4F97D20C000F44908600846006815
:10208000FEF786FB0120E4490883FEF7BFFBE12051
:102090004002EF490860FEF7B7FAE6490863ED48E9
:1020A000C088DD49088201200882FEF7B1FE0121C7
:1020B000E948FEF7D0FC0421E748FEF7CCFCE648EF
:1020C000FEF7E3FC01210903E348FEF7C4FC6421A9
:1020D000E148FEF7CFFDFEF7FFFD0121DF48FEF7E7
:1020E000BAFC0421DD48FEF7B6FCDC48FEF7CDFC67
:1020F000D948FEF7C4FCD948FEF7C1FCD648FEF724
:10210000AEFCD648FEF7ABFC01208004CD494969FE
:102110000143CC4A5161114649690140089100BF11
:1021200000BF182120A8FEF745F8012000032090E9
:102130000120219003202290002023900120249050
:1021400020A9C748FEF798FB01210903C448FEF700
:102150001EFC0120C003209001202190032022902A
:10216000002023900120249020A90920C006FEF71A
:1021700083FB082020900120219003202290002042
:1021800023900120249020A9B548FEF775FB20205C
:102190002090012021900320229001202390249060
:1021A00020A9AF48FEF768FB0121C9030920C0063A
:1021B000FEF7EFFB0821AA48FEF7EBFB2021A84819
:1021C000FEF7E7FBFFF726FB5621A6480170012426
:1021D00001201F90A4481E90A4481E99FDF798FF67
:1021E000401E1D9032201C901C991D9840181B9079
:1021F0001C991D98401A1A901D9D002019900120CD
:1022000018909B48017810A801739948417810A84C
:1022100041739748817810A881739548C17810A8B8
:10222000C1739348017910A801729148417910A8AF
:1022300041728F48817910A881728D48C17910A8A8
:10224000C1728B48017A10A801718948417A10A89F
:1022500041718748817A10A881718548C17A10A898
:10226000C1710021017055214170FF218170002151
:10227000C17000BF00200A90099026E2F105C80F46
:10228000FFF784F8761CFFF7C5FA0FA8FFF708FAE6
:1022900008A8017F0E91007EC009002807D008A879
:1022A000007DC009002802D10C98401C0C9008A8A1
:1022B000007E0007C00F002808D008A8007D000796
:1022C000C00F002802D10C98401E0C9008A8007E78
:1022D0004007C00F002806D008A8007D4007C00FA7
:1022E000002800D17F1E08A8007E4006C00F0028ED
:1022F00006D008A8007D4006C00F002800D17F1C32
:1023000008A8007E8006C00F00281ED008A8007D07
:102310008006C00F002818D10A98002801D101209A
:1023200000E000200A900A98002807D000244A48BC
:10233000FEF7A5FB4948FEF7A2FB06E0002446484D
:10234000FEF78DFB4548FEF78AFB08A8007E800754
:10235000C00F002814D008A8007D8007C00F0028F7
:102360000ED10998002801D1012000E00020099039
:102370000998002802D00120199001E0002019904E
:102380000E980D90FEF740F908900A98002811D198
:102390003748C17B10A801733548C17B10A8417331
:1023A0003348017810A8817331482030417810A853
:1023B000C1730FE02E48C17B10A8C1732C488178EF
:1023C00010A881732A48017E10A84173284801781B
:1023D00010A8017310A8017B0176417B8176817B77
:1023E0000177C17B8177FEF70FF90790089907986D
:1023F000401A069000200590059F1D48817A10A87C
:1024000001720A213846FDF783FE1948415C10A885
:1024100041720A2138462DE0F00600209007002086
:10242000100700208C010020D40800209408002010
:10243000DC010020CC0400209F86010080F7FF1FF4
:102440004000002000100240102700001C00002067
:10245000B40000202C020020002C0140004001406C
:10246000000400484C060020606D0000006CDC0297
:102470001E1D0008FDF74CFE0A210190FDF748FEE5
:1024800010319248415C10A88172642F0CDB6421EA
:102490003846FDF73DFE0A210190FDF739FE8B48D5
:1024A000415C10A8C17203E008A8017F10A8C172A6
:1024B00010A8017A4174417AC174817A4175C17A58
:1024C000C1750020049004980B900A210B98FDF729
:1024D0001FFE7E48415C10A801710A210B98FDF790
:1024E00017FE0A210190FDF713FE7848415C10A801
:1024F000417164210B98FDF70BFE0A210190FDF755
:1025000007FE7248415C10A881717D21C9000B98BB
:10251000FDF7FEFD0A210190FDF7FAFD6B48415CD5
:1025200010A8C171017901744179817481790175B3
:10253000C17981757006C10E01208840401E03904C
:102540002046E117C90E09184911091DCA06D20E05
:1025500001219140491E03910398C1B210A8017056
:1025600003980004010E10A8417003980002010EA8
:1025700010A881708178C176417841770178C17760
:10258000102214A90020FFF7E7F86420FEF707F8EF
:102590001998002829D0F007C00F002825D06D1EFB
:1025A0001A98854200DC1B9D29464948FEF766FBC8
:1025B00029464848FEF762FB681CC20F01901018BC
:1025C0004010411E4348FEF753FB681CC20F12180F
:1025D0005210511E3F4A116400BFC20F01901018E3
:1025E0004010411E3A48FEF743FB0A9800281BD0D2
:1025F0001898002818D0B007800F022814D11F980F
:10260000012807D13448844201DA641C08E0002024
:102610001F9005E0012C01DD641E01E001201F90E8
:1026200021462B48FEF726FBFDF722FE0920C006B7
:10263000FEF7AAF90290029881B22848018628483C
:10264000FEF7A2F90290029881B2244841862548FB
:10265000FEF79AF90290029881B2204881862248BA
:10266000FEF792F90290029881B21C48C186FDF7EC
:10267000CBFF1E4908601E480068002802D00021D8
:102680001C4801801C48007BC006C00E02281BD1DC
:102690001748006800280FD0002016490880174806
:1026A0000068002810D112480168144801601448DD
:1026B00001681448016007E010480068002803D052
:1026C0000B4800680D49086000BFD7E51E1D0008D3
:1026D00000400140002C0140BB0200008C0600209D
:1026E0000004004800080048000C0048CC0000200E
:1026F00094000020AC020020CC04002098000020B0
:102700002C0000209C0000200000000000000000C1
:1027100000000000000000000000000000000000B9
:102720000100000010270000000000000000000071
:102730000000000000000000000000000000000099
:102740000000000000000000000000000000000089
:102750000100000000000000000000000302000073
:102760000101010000000000000000000000000066
:102770000000000000000000000000000000000059
:102780000000000000000000000000000000000049
:102790000000000000000000000000000000000039
:1027A0000100000000000000FFFFFFFF000000002C
:1027B00000000000000000000100000000C2010055
:1027C00040420F0000000000000000000000000078
:1027D00000000000000000000000000000000000F9
:1027E000000000000000000000000000001BB70017
:0427F00000000000E5
:04000005080000B53A
:00000001FF
